:10000000A6C00000B6C00000B4C00000B2C000002E
:10001000B0C00000AEC00000ACC00000AAC000002C
:10002000A8C00000A6C000000C94E208A2C0000016
:10003000A0C000009EC000009CC000009AC000004C
:1000400098C0000096C0000094C0000092C000005C
:1000500090C000008EC000008CC000008AC000006C
:1000600088C0000086C0000084C0000082C000007C
:1000700080C0000012C300007CC000007AC00000F5
:1000800078C0000076C0000074C0000072C000009C
:1000900070C000006EC000006CC000006AC00000AC
:1000A00068C0000066C0000064C0000012010002C9
:1000B00000000020EB0313200010010200010902E0
:1000C0002900010100803209040000020300000041
:1000D00009211101000122350007058103080014E0
:1000E000070502030800140C03410054004D0045AD
:1000F000004C0022034100560052002000550053DE
:10010000004200200048004900440020004400450F
:10011000004D004F000403090406FFFF0901A1017F
:1001200009020903150026FF0075089508810209D8
:10013000040905150026FF007508950891020906B7
:100140000907150026FF0075089504B102C01124A7
:100150001FBECFEFDAE0DEBFCDBF81E011E0A0E04F
:10016000B1E001C01D92A832B107E1F7FCD50C94B3
:10017000FD0946CFE8EDF0E080818F7780838081B4
:1001800080688083808180618083808181608083BA
:10019000789408958091D80080628093D80082B7C7
:1001A000807F82BF82B78A6482BF82E089BD09B442
:1001B00000FEFDCF8091D8008F7D8093D800809184
:1001C000E0008E7F8093E0008091E000877F809345
:1001D000E0008091E20081608093E2008091E20083
:1001E00088608093E200789447C080910001882362
:1001F00069F48091D90080FF09C08091D80080689F
:100200008093D80081E080930001C4DF80911001C9
:100210009091110190FF10C08091100190911101F7
:100220009E7F909311018093100181E08093EA00FA
:100230001092EA00109224011092E9008091E800E7
:1002400083FF01C099C508959091EB009160909350
:10025000EB008093EC008091ED008270862B809300
:10026000ED008091ED0082608093ED008091EE00C2
:10027000881F8827881F08951092E9008091EB005D
:1002800080FF02C080E008951092E90082E060E201
:10029000DBCF8330F1F4613059F0613018F0623017
:1002A000C1F40CC084E08093250185E191E00BC08E
:1002B0008CE08093250187EE90E005C082E2809378
:1002C000250183EF90E0909327018093260181E040
:1002D000089580E00895DF93CF9300D000D0CDB78C
:1002E000DEB78091F1008B838091F1008C8385E3F0
:1002F0008093250189E191E0909327018093260165
:100300008091F10089838091F1008A838091E800D7
:10031000877F8093E80089819A818633910528F050
:100320004091250129E131E01CC080932501F8CFDF
:100330008091E80080FFFCCFF90190E00AC0542FC3
:100340005150903249F09F5F84918093F100319633
:10035000452F9F01442399F78091E8008E7F809379
:10036000E800442359F08091E80082FFE1CF309308
:100370002701209326014093250106C030932701D1
:1003800020932601109225018091E80082FFFCCF86
:100390008091E8008B7F8093E8008091E8008F7760
:1003A0008093E8000F900F900F900F90CF91DF9106
:1003B00008958091E800877F8093E8008091E800AD
:1003C0008E7F8093E8008091E80082FFFCCF8091CF
:1003D000E8008B7F8093E8008091E8008F7780931E
:1003E000E8008091E8008E7F8093E8000895DF9315
:1003F000CF9300D0CDB7DEB78091F1008983809193
:10040000F1008A838091E800877F8093E800609301
:1004100003018091E8008E7F8093E8008091E800DE
:1004200080FFFCCF0F900F90CF91DF910895DF9365
:10043000CF9300D000D0CDB7DEB78091F1008B8391
:100440008091F1008C838091F10089838091F1008B
:100450008A838091E800877F8093E80089819A8170
:10046000892B49F0809103018093F1008091E8008D
:100470008E7F8093E8008091E80082FFFCCF80911E
:10048000E8008B7F8093E8008091E8008F7780936D
:10049000E8000F900F900F900F90CF91DF9108958B
:1004A0008091E800877F8093E8008091E8008E7F4C
:1004B0008093E8008091E80082FFFCCF8091F100FA
:1004C000853579F48091F1008A3A59F48091F100F0
:1004D000853539F48091F1008A3A19F481E08093EE
:1004E00002018091E8008B7F8093E8008091E80012
:1004F0008F778093E8008091E8008E7F8093E800FA
:100500008091E80080FFFCCF0895DF93CF9300D067
:1005100000D0CDB7DEB78091F1008B838091F100E0
:100520008C8389E08093250180ED90E090932701F2
:10053000809326018091F10089838091F1008A8364
:100540008091E800877F8093E80089819A818A30D2
:10055000910528F04091250120ED30E01CC08093EA
:100560002501F8CF8091E80080FFFCCFF90190E0F1
:100570000AC0542F5150903249F09F5F849180936C
:10058000F1003196452F9F01442399F78091E800AF
:100590008E7F8093E800442359F08091E80082FF29
:1005A000E1CF30932701209326014093250106C017
:1005B0003093270120932601109225018091E800B5
:1005C00082FFFCCF8091E8008B7F8093E8008091D0
:1005D000E8008F778093E8000F900F900F900F90B6
:1005E000CF91DF9108952091F1009091F100813831
:1005F00059F4663029F5913219F0923209F502C0AA
:1006000084DF1CC068DE1AC0813291F4693019F0B1
:100610006A30B1F409C0923019F0933089F402C005
:10062000C8DE0CC03DDF0AC0822F692FE0DE06C0A5
:10063000813A31F4623021F4822FF9DE81E00895AD
:1006400080E008950F931F9309EE10E081E0F80118
:10065000808381EC60E0F8DD82E0F801808380EC4B
:1006600060E0F2DD1F910F910895BFD622D3FDCF38
:10067000BFD643C3FDDFF9CF81E480937C001092A5
:100680007B00EAE7F0E086E0808386E980838EECF9
:10069000808383E380937E0008951F920F920FB6AC
:1006A0000F9211242F938F939F9380911301843085
:1006B00009F455C0853050F4813071F18130C8F0B3
:1006C000823099F1833009F08DC042C0873009F43F
:1006D0006BC0883038F4853009F450C0863009F09A
:1006E00081C053C0883009F467C0893009F07AC0EE
:1006F00072C080917800909179002FE420937C0063
:1007000010927B0096958795969587959093180102
:100710008093170181E006C081E480937C001092F1
:100720007B0082E0809313015DC0809178009091FE
:1007300079002FE420937C0010927B00969587959A
:100740009695879590931A018093190183E0EACFDB
:1007500084E480937C0010927B0084E0E3CF80915E
:1007600078009091790090931C0180931B018FE495
:1007700080937C0010927B0085E0D4CF85E4809349
:100780007C0010927B0086E0CDCF80917800909124
:10079000790090931E0180931D018FE480937C006B
:1007A00010927B0087E0BECF87E480937C0080E2DC
:1007B00080937B0088E0B6CF80917800909179009B
:1007C0009093200180931F018FE480937C0010920E
:1007D0007B0089E0A7CF80E480937C0010927B00AF
:1007E000109213018EEC80937A009F918F912F913C
:1007F0000F900FBE0F901F90189592E09093E90014
:100800008091E80082FFD5C18091F1003091F10024
:100810002091F1004091F1005091F1005091F100D0
:100820005091F1005091F1008C3409F4A1C08D3445
:1008300040F48334B1F1843469F0813409F0AFC1FC
:100840005EC1823509F469C08335F1F1803509F064
:10085000A6C15CC1832F30FF02C05C9A01C05C98C6
:1008600081FF02C05E9A01C05E9882FF02C05F9A5B
:1008700001C05F9883FF02C02C9A01C02C9884FFAE
:1008800002C02D9A01C02D9885FF02C02E9A01C08A
:100890002E9886FF02C0469A01C0469837FFD3C003
:1008A00097C0832F30FF02C02F9A01C02F9881FF7D
:1008B00002C02B9A01C02B9882FF02C0299A01C066
:1008C000299883FFA0C064C0303309F465C0313378
:1008D00009F466C0323309F467C0333309F468C0E1
:1008E000343309F469C0353309F46AC0363309F486
:1008F0006BC0373309F46CC03435F1F1363409F488
:100900003FC0393409F444C03335F1F1323509F4CC
:1009100063C0353409F465C042C1303309F477C08F
:10092000313309F478C0323309F479C0333309F430
:100930007AC0343309F47BC0353309F47CC03633D4
:1009400009F47DC0373309F47EC0343509F44FC053
:10095000363409F450C0393409F455C0333509F43C
:100960004EC0323509F473C0353409F475C017C16F
:100970003E34C9F5213011F42F9A11C1223011F4FF
:100980002B9A0DC1233011F4299A09C1243011F496
:100990002A9A05C1253011F45C9A01C1263011F460
:1009A0005E9AFDC0273011F45F9AF9C0283011F427
:1009B0002C9AF5C0293011F42D9AF1C02A3011F487
:1009C0002E9AEDC02B3011F4469AE9C02C3011F468
:1009D000479AE5C02D3011F4289AE1C02E3009F075
:1009E000DEC0769ADCC03634C9F5213011F42F9878
:1009F000D6C0223011F42B98D2C0233011F429989C
:100A0000CEC0243011F42A98CAC0253011F45C9865
:100A1000C6C0263011F45E98C2C0273011F45F982A
:100A2000BEC0283011F42C98BAC0293011F42D988A
:100A3000B6C02A3011F42E98B2C02B3011F446986B
:100A4000AEC02C3011F44798AAC02D3011F428986C
:100A5000A6C02E3009F0A3C07698A1C0343509F0A5
:100A60009EC0213019F485B1805824C0223019F479
:100A700085B198E01EC0233011F485B11AC024302E
:100A800019F485B1822716C0253019F48BB190E195
:100A900004C0263021F48BB190E4892704C02730AC
:100AA00021F48BB180588BB97AC0283029F485B1F4
:100AB00090E1892785B973C0293019F485B190E296
:100AC000F8CF2A3019F485B190E4F3CF2B3021F41C
:100AD00088B190E4892704C02C3021F488B1805873
:100AE00088B95DC02D3019F485B191E0E2CF2E3088
:100AF00009F055C08EB190E489278EB950C03434C6
:100B000009F04DC081E08093160149C0942F80E028
:100B1000AC01420F511D3134A9F48FEF93E0909353
:100B20008700809386008091800080688093800099
:100B300083E180938100109282005093890040935A
:100B400088002DC03234A9F48FEF93E09093870092
:100B5000809386008091800080628093800083E192
:100B6000809381001092820050938B0040938A0002
:100B700016C03334A1F48FEF93E0909387008093F5
:100B800086008091800088608093800083E180935C
:100B900081001092820050938D0040938C008091D0
:100BA000E8008B7F8093E8008091E8008F77809346
:100BB000E800089581E08093E9008091E80085FFD6
:100BC00077C029B120952170499B2E5F4D9B2C5FEA
:100BD000629B285F7F9B205F7E9B205E809114013B
:100BE00090911501019690931501809314018091C5
:100BF0001601813079F510921601109215011092AC
:100C000014012093F100809117018093F1008091ED
:100C100019018093F10080911B018093F100809174
:100C20001C018093F10080911D018093F10080915F
:100C30001E018093F10080911F018093F10080914B
:100C4000E8008E7F8093E8008091E8008F778093A2
:100C5000E800089580910501281751F120930501BE
:100C60002093F100809117018093F1008091190188
:100C70008093F10080911B018093F10080911C0111
:100C80008093F10080911D018093F10080911E01FD
:100C90008093F10080911F018093F1008091E80022
:100CA0008E7F8093E8008091E8008F778093E80042
:100CB000089580912401882311F09FDD7BCF089552
:100CC000809104018F5F8093040108958AE090E78A
:100CD000FC018491EBE0F0E73491ECE0F0E7249143
:100CE000EDE0F0E794918C3231F4313121F42C3283
:100CF00011F4923209F037C008950F931F9385B70E
:100D0000806885BF85B7806885BF85B7806885BFE7
:100D100085B7806885BF85B7806885BF8FEF84B948
:100D200080EC87B980ED8AB980E48DB910BA15B826
:100D30008FE388B98FE28BB98FEB8EB98CEC81BBD6
:100D400000E810E0F8011082C1DF10921501109246
:100D500014011092130190DCF80110821092160118
:100D60001F910F910895E7EDF0E08081816080830D
:100D700081DC80E090E00895DF93CF9300D0CDB781
:100D8000DEB78091E8008B7F8093E8009091F100BE
:100D900090930F016091F1006630F9F0673068F4CC
:100DA000613009F41AC1613008F496C1633009F466
:100DB0004EC1653009F0F3C1D5C0693009F4F4C003
:100DC0006A3020F4683009F0EAC1AFC06A3009F433
:100DD000B8C16B3009F0E3C1D1C1903809F0A2C0AD
:100DE000109207016091F1008091F100813019F0BB
:100DF000823089F406C082E1809325018CEA90E07C
:100E000005C089E2809325018EEB90E09093270145
:100E10008093260104C03DDA882309F4C4C180917F
:100E2000F1008091F1008091F10089838091F100BF
:100E30008A838091E800877F8093E80029813A8146
:100E40008091250190E08217930758F48F7190707C
:100E5000892B21F481E08093070105C010920701DE
:100E600002C0209325018091E8008F7E8093E800E6
:100E700020912601309127014091250122C08091C7
:100E8000E80084FF03C0F90190E00FC08091E80002
:100E900080FFF5CFF8CF542F5150903249F09F5F2B
:100EA00084918093F1003196452F9F01442399F757
:100EB0008091E80084FD12C08091E8008E7F8093CD
:100EC000E800442339F4209326013093270110923F
:100ED00025010AC08091E80084FFD8CF2093260125
:100EE000309327014093250180910701813069F4F7
:100EF0008091E80084FD09C08091E80080FFFCCF6C
:100F00008091E8008E7F8093E8008091E80084FF64
:100F1000FCCF8091E8008F7E8093E8008091E8000C
:100F20008B7F49C1892F66E027C19038C1F4809139
:100F3000E800877F8093E800809124018093F1008E
:100F40008091E8008E7F8093E8008091E8008F77A1
:100F50008093E8008091E80082FFFCCF02C1892FD6
:100F600068E00AC19923E9F49091F1008091E300CF
:100F70009F778078982B9093E3008091E800877F9B
:100F80008093E8008091E8008E7F8093E800809154
:100F9000E80080FFFCCF8091E30080688093E3004D
:100FA0000CC1892F65E0E8C09923A1F49091F1006C
:100FB000923008F0F8C08091E800877F8093E800C5
:100FC000909324018091E8008E7F8093E800892F20
:100FD00039DBF3C0892F69E0CFC09330A8F599239E
:100FE00009F441C0913009F4DEC08091F100909184
:100FF000F100882309F0D7C0E091F100EF77E0938A
:10100000E9008091EB0080FF61C0EE23B1F0809198
:10101000EB0080618093EB0081E090E00E2E02C037
:10102000880F991F0A94E2F78093EA001092EA0071
:101030008091EB0088608093EB001092E900F0E073
:10104000E85FFE4F108239C0892F61E095C0933070
:1010500008F03FC0913009F4A6C0913020F09230E2
:1010600009F0A1C003C08091F1009DC08091F10002
:101070009091F100882309F096C0E091F100EF779C
:1010800051F48091EB0080628093EB008091E80046
:10109000877F8093E800E093E9008091EB0080FF78
:1010A00015C08091EB0080628093EB001092E90004
:1010B000F0E0E85FFE4F81E080838091E800877F69
:1010C0008093E8008091E8008E7F75C01092E9005F
:1010D0006AC0892F63E050C0892F8058833070F533
:1010E0008091F1008091F100E091F100913829F0B8
:1010F000923859F0903809F056C08091E800877F07
:101100008093E8001092F1000DC08091E800877F85
:101110008093E800F0E0EF77F070E85FFE4F8081A9
:101120008093F1001092F1008091E8008E7F80930F
:10113000E8008091E80082FFFCCF13C0892F60E0B7
:101140001BC09138B9F48091E800877F8093E80054
:101150008091E8008E7F8093E8008091E80082FF14
:10116000FCCF8091E8008B7F8093E8008091E800BD
:101170008F7721C0892F6AE036DA1FC09130E9F4F9
:101180008091E800877F8093E8008091E8008E7F5F
:101190008093E8008091E80080FFFCCF0EC0892F8B
:1011A00022DA882351F48091EB0080628093EB0077
:1011B0008091E800877F8093E8000F900F90CF9197
:1011C000DF9108951F920F920FB60F9211242F9363
:1011D0003F934F935F936F937F938F939F93AF93BF
:1011E000BF93EF93FF938091DA0080FF31C080912D
:1011F000D80080FF2DC08EEF8093DA008091D90057
:1012000080FF19C081E080930001809110019091CE
:101210001101826090931101809310018091E2008E
:1012200088608093E2000E94CA008091E0008E7F77
:101230008093E0000DC01092000110922401809173
:10124000100190911101846090931101809310011D
:101250008091E10082FF08C08091E20082FF04C01B
:101260008BEF8093E1002CDD8091E10080FF29C0AD
:101270008091E20080FF25C081E0809301018FEE24
:101280008093E10080911001909111018062909310
:101290001101809310018EEF8093E1008091E200B4
:1012A00080618093E2008091E2008F7D8093E20074
:1012B0008091D80080628093D80089B58D7F89BDE8
:1012C00019BC8091E10084FF47C08091E20084FF57
:1012D00043C009B400FC0BC082B7807F82BF82B7D5
:1012E0008A6482BF82E089BD09B400FEFDCF80918F
:1012F000D8008F7D8093D8009FEE9093E10080917D
:101300000101882349F18091E20080628093E2002C
:101310008091E20088608093E2009093E1008091E8
:10132000E2008F7E8093E200809110019091110184
:10133000806490931101809310018091E20081609C
:101340008093E2008091E20080628093E2008091CD
:10135000E20088608093E2008091E10085FF1CC07C
:101360008091E20085FF18C0109201018091E20097
:101370008F7E8093E2008FED8093E1008091E20008
:101380008F7D8093E200809110019091110180681F
:1013900090931101809310018091E10083FF14C0AC
:1013A0008091E20083FF10C01092230187EF8093A9
:1013B000E1000E943C018091100190911101916027
:1013C0009093110180931001FF91EF91BF91AF9124
:1013D0009F918F917F916F915F914F913F912F914D
:1013E0000F900FBE0F901F9018950C94F500089564
:0E13F0000E94BA00109223010895F894FFCFD6
:00000001FF
